:0200000480007A
:100000006F008004732F2034930F80006308FF0378
:10001000930F90006304FF03930FB0006300FF038E
:10002000130F000063040F0067000F00732F2034CC
:1000300063540F006F00400093E19153171F0000BD
:1000400023223FFC6FF09FFF93000000130100008C
:10005000930100001302000093020000130300004C
:100060009303000013040000930400001305000034
:10007000930500001306000093060000130700001C
:100080009307000013080000930800001309000004
:1000900093090000130A0000930A0000130B0000EC
:1000A000930B0000130C0000930C0000130D0000D4
:1000B000930D0000130E0000930E0000130F0000BC
:1000C000930F0000732540F16310050097020000B4
:1000D000938202017390523073500018970200000F
:1000E00093824202739052309B021000939252030B
:1000F0009382F2FF7390023B9302F0017390023AF5
:100100007350403097020000938242017390523046
:10011000735020307350303093010000970200007C
:10012000938282EE73905230130510001315F5017F
:10013000635C05000F00F00F930110009308D005D9
:10014000130500007300000093020000638A0200A0
:1001500073905210B7B200009B82921073902230BD
:100160007350003097020000938242017390123462
:10017000732540F173002030B700008013010000A8
:100180003BD72000B70300809301200063187760FD
:10019000B7000080130110003BD72000B7030040D8
:1001A00093013000631C775EB7000080130170007C
:1001B0003BD72000B7030001930140006310775E36
:1001C000B70000801301E0003BD72000B703020016
:1001D000930150006314775CB70000809B8010008F
:1001E0001301F0013BD7200093031000930160003E
:1001F0006316775A9300F0FF130100003BD72000ED
:100200009303F0FF93017000631A77589300F0FF97
:10021000130110003BD72000B70300809B83F3FF3E
:1002200093018000631C77569300F0FF1301700068
:100230003BD72000B70300029B83F3FF930190009C
:10024000631E77549300F0FF1301E0003BD72000BA
:10025000B70304009B83F3FF9301A000631077545E
:100260009300F0FF1301F0013BD72000930310002F
:100270009301B00063147752B72021219B801012A4
:10028000130100003BD72000B72321219B831312C9
:100290009301C00063147750B72021219B80101276
:1002A000130110003BD72000B79390109B830309E4
:1002B0009301D0006314774EB72021219B80101248
:1002C000130170003BD72000B74342009B832324D7
:1002D0009301E0006314774CB72021219B8010121A
:1002E0001301E0003BD72000B78300009B83434805
:1002F0009301F0006314774AB72021219B801012EC
:100300001301F0013BD7200093030000930100018B
:1003100063167748B72021219B801012130100FE3D
:100320003BD72000B72321219B8313129301100197
:1003300063167746B72021219B801012130110FE0F
:100340003BD72000B79390109B83030993012001B2
:1003500063167744B72021219B801012130170FE91
:100360003BD72000B74342009B83232493013001F5
:1003700063167742B72021219B8010121301E0FE03
:100380003BD72000B78300009B8343489301400183
:1003900063167740B72021219B8010121301F0FFD4
:1003A0003BD7200093030000930150016318773E70
:1003B000B720F1FF9B8050349390C00093808067FA
:1003C000130100003BD72000B75334129B8383678F
:1003D0009301C0026314773CB720F1FF9B80503437
:1003E0009390C00093808067130140003BD72000AA
:1003F000B74323019B8373569301D0026310773A6E
:10040000B72009009B8050349390C0009380806790
:10041000130100003BD72000B75334929B838367BE
:100420009301E002631C7736B72009009B805034AB
:100430009390C00093808067130140003BD7200059
:10044000B74323099B8373569301F00263187734F3
:10045000B700008013017000BBD02000B70300017B
:1004600093016001639C7032B70000801301E000CB
:100470003BD12000B7030200930170016310713279
:1004800093007000BBD01000930300009301800123
:100490006396703013020000B700008013017000F3
:1004A0003BD7200013030700130212009302200021
:1004B000E31452FEB7030001930190016310732E01
:1004C00013020000B70000801301E0003BD72000BA
:1004D0001300000013030700130212009302200010
:1004E000E31252FEB70302009301A0016318732ABE
:1004F00013020000B70000801301F0013BD7200079
:100500001300000013000000130307001302120081
:1005100093022000E31052FE930310009301B001F8
:10052000631E732613020000B700008013017000E1
:100530003BD720001302120093022000E31652FE64
:10054000B70300019301C001631A7724130200006E
:10055000B70000801301E000130000003BD720002B
:100560001302120093022000E31452FEB7030200AC
:100570009301D0016314772213020000B7000080BA
:100580001301F00113000000130000003BD720000E
:100590001302120093022000E31252FE9303100094
:1005A0009301E001631C771E13020000B700008076
:1005B00013000000130170003BD72000130212004B
:1005C00093022000E31452FEB70300019301F001EF
:1005D0006316771C13020000B700008013000000B0
:1005E0001301E000130000003BD7200013021200AB
:1005F00093022000E31252FEB703020093010002AF
:10060000631E771813020000B7000080130000007B
:10061000130000001301F0013BD720001302120069
:1006200093022000E31252FE930310009301100284
:10063000631677161302000013017000B7000080E4
:100640003BD720001302120093022000E31652FE53
:10065000B703000193012002631277141302000014
:100660001301E000B7000080130000003BD720001A
:100670001302120093022000E31452FEB70302009B
:1006800093013002631C7710130200001301F00184
:10069000B700008013000000130000003BD72000CB
:1006A0001302120093022000E31252FE9303100083
:1006B000930140026314770E1302000013017000CF
:1006C00013000000B70000803BD720001302120087
:1006D00093022000E31452FEB7030001930150027D
:1006E000631E770A130200001301E00013000000EC
:1006F000B7000080130000003BD720001302120057
:1007000093022000E31252FEB7030200930160023D
:1007100063167708130200001301F00113000000B4
:1007200013000000B70000803BD720001302120026
:1007300093022000E31252FE930310009301700213
:10074000631E77049300F0003B51100093030000F8
:100750009301800263147104930000023BD10000F6
:100760009303000293019002631A7102BB500000D0
:10077000930300009301A002639270029300004073
:10078000371100001B0101803BD0200093030000C3
:100790009301B00263147000631030020F00F00F79
:1007A000638001009391110093E111009308D0053B
:1007B00013850100730000000F00F00F930110007B
:1007C0009308D0051305000073000000731000C0EB
:1007D0000000000000000000000000000000000019
:1007E0000000000000000000000000000000000009
:0C07F000000000000000000000000000FD
:1010000000000000000000000000000000000000E0
:1010100000000000000000000000000000000000D0
:1010200000000000000000000000000000000000C0
:1010300000000000000000000000000000000000B0
:081040000000000000000000A8
:040000058000000077
:00000001FF
